:104DB100754906123280202F04E52E70F91232C98E
:104DC10075490612324080E822754904123280E5A5
:104DD1002E70FC1232C97549041232407F01122A29
:104DE100C27E007FFF8F05124BADDFF97E007FFF92
:104DF100900000C007124BEAEFF0A3D007DFF422C6
:104E0100754901123280E52E70C51232C97549010A
:104E110012324022754A01122AC27808302DFDE56E
:0B4E21003C2430122A93C22DD8EA2254
:10250A00758400854ED2854FD37584018550D28556
:10251A0051D3E4F54FF54E30080685524E85534F98
:10252A0030090CE54E2554F54EE54F3555F54F303B
:10253A000A10E5328533F0A4254EF54EE5F0354F05
:10254A00F54F300B10E50A8536F0A4254EF54EE519
:10255A00F0354FF54F300C10E5118535F0A4254EB6
:10256A00F54EE5F0354FF54FE4F551F550301010C2
:10257A00855250855351E553C3953A4003853A51E4
:10258A00301116E555C395394003853A55E550256E
:10259A0054F550E5513555F551301210E532853371
:1025AA00F0A42550F550E5F03551F551301310E5FA
:1025BA000A8536F0A42550F550E5F03551F551302D
:1025CA001410E5118535F0A42550F550E5F0355184
:1025DA00F551301510E5188534F0A42550F550E56D
:1025EA00F03551F551301610E5278538F0A42550FD
:1025FA00F550E5F03551F551301710E5288537F0DB
:10260A00A42550F550E5F03551F551E551C3953BF8
:10261A004003853B512290268730310312264230EF
:07262A003203122652303486
:1026310003122676303303122675303503122686AF
:1026410022E50B2509F50BE50C3508F50C93F50A88
:1026510022E512250EF512E513350DF51393C3137B
:10266100F8E5142510F514E515350FF51593C31389
:1026710028F5112222E5192517F519E51A3516F560
:102681001A93F51822227F8285888C8F9295989BC8
:102691009EA1A4A7AAADB0B3B6B9BBBEC1C3C6C9FA
:1026A100CBCED0D3D5D7D9DCDEE0E2E4E6E7E9EB67
:1026B100EDEEF0F1F2F4F5F6F7F8F9FAFBFCFCFDBA
:1026C100FDFEFEFEFEFEFEFEFEFEFEFDFDFCFCFB33
:1026D100FAFAF9F8F7F6F4F3F2F0EFEDECEAE8E7DD
:1026E100E5E3E1DFDDDBD8D6D4D1CFCDCAC8C5C2A1
:1026F100C0BDBAB7B4B2AFACA9A6A3A09D9A979436
:10270100908D8A8784817E7A7774716E6B68656239
:102711005F5C595653504D4A4744423F3C39373428
:10272100322F2D2A282624211F1D1B191816141299
:10273100110F0E0C0B0A080706050404030202011F
:10274100010000000000000000000001010202037E
:102751000405060708090A0B0D0E101113151618AA
:102761001A1C1E20222427292B2E303335383A3DBE
:10277100404245484B4E515456595C606366696C02
:062781006F7275787B7F8A
:1029F000D2F4C2F5C2F675840F85F0C8122820748F
:102A000003122A3F1228147403122A3F1227F712C6
:102A100027F77403122A3F1227F77402122A3F1273
:102A200027F77428122AAB7406122AAB740E122AE6
:102A3000AB7401122AAB1228147480122AAB22C084
:102A400000A2E092F3A2E192F2A2E292F1A2E3925A
:102A5000F0D2F475840F85F0C8C2F47830D8FE85C2
:102A6000F0C87830D8FED00022C00075840FA2E4F0
:102A700092F3A2E592F2A2E692F1A2E792F0D2F4EA
:102A800085F0C8C2F47830D8FE85F0C87830D8FE1A
:102A9000D00022EF75840FD2F5C2F685F0C8122A55
:102AA000691227F7122A3F1227F72275840FC2F501
:102AB000C2F685F0C8122A691227F7122A3F122798
:102AC000F722EF14A2E492E6C2E4D2E7122AAB2284
:102AD000740F122AAB22740D122AAB227F01122A24
:102AE000C278107F20122A93D8F9227F11122AC2AD
:102AF00078107F20122A93D8F9227F01122AC278F7
:102B0000207F20122A93D8F922C0077F018004C0B9
:102B1000077F11122AC2D007C082C083C007EF7599
:102B2000F010902B3A1228387810E493FF122A9371
:092B3000A3D8F7D007D083D082AE
:102B3900222020202020202020202020202020208A
:102B49002030313233343536373839414243444500
:102B590046202020525334323220544553542020E9
:102B69002020202052533233322054455354202000
:102B79002020205445535420204641494C454420A7
:102B8900202020544553542020504153534544207C
:102B9900202020454550524F4D2054455354202064
:102BA90020204155582052454C41592054455354F1
:102BB9002020205055534820544F2054414C4B203D
:102BC9002054455354203320434841522F535542F2
:102BD900205445535420464958454420535452499A
:102BE9004E54455354205641524942205354524958
:102BF9004E464143544F52592044454641554C5441
:102C09002050524F4752414D4D494E47204D4F4458
:102C19004553494D504C455820524550454154451E
:102C2900522020205245434F5244494E47202020EC
:012C3900207A
:104BAD00758400D2C2C2C6D2C6C2C4D2C5C2C33079
:104BBD00C3FD74A0F5C2C2C5C2C330C3FD8EC2C24F
:104BCD00C330C3FD8FC2C2C330C3FD8DC2C2C3305B
:104BDD00C3FDD2C4C2C320C4FD12281422758400A3
:104BED00C2C3D2C530C3FD74A0F5C2C2C5C2C330A5
:104BFD00C3FD8EC2C2C330C3FD8FC2C2C330C3FD5D
:104C0D00C2C4D2C5C2C330C3FD74A1F5C2C2C5C2F0
:104C1D00C330C3FDC2C2C2C330C3FD85C207D2C4F7
:064C2D00C2C320C4FD22F9
:0800030002303700000000008C
:08000B00023038000000000083
:080013000231AF000000000003
:08001B003200000000000000AB
:09002300320000000000000000A2
:08002B0002303B000000000060
:08003300320000000000000093
:0A003B003200000000000000000089
:0900430032000000000000000082
:08004B0032000000000000007B
:08005300320000000000000073
:08005B0002309A0000000000D1
:08006300320000000000000063
:08006B000230B80000000000A3
:08007300023041000000000012
:08007B000231B000000000009A
:080083000230970000000000AC
:08008B0032000000000000003B
:100093000231CE000000000000000000000000005C
:1000A3003275FF0775FFDE75FFAD75840F75E107C8
:1000B30075E20475E34475840F75A43575A5097558
:1000C300A6FF75A7FF759CFF759D00759E00759F24
:1000D300F075D8FF75E8FF75F80F75AD0F758401DE
:1000E30075893075888F75840275893075888F7529
:1000F300840F758A80758C67780874FF0000000090
:100103000000000000000000D5E0F1D8EDE58C30E0
:10011300E7FB759701758A0043890475840075B7F9
:100123001075840F438901758D01758F01758E02DA
:100133007480D5E0FD438902E58930E4FB759702BD
:1001430075840075D10775840075BB0175BA007598
:10015300BCF075C70075C60075C5FF75C4FF75E8AB
:100163008175840275BB0475BA0075BCF175C60050
:1001730075C4FF75E88875840075D484758401752A
:10018300D484758400C2F8759A47759D1A43F8099B
:1001930075870075840075B90075A90075910075A0
:1001A300985075840175981075840075C04075C3A7
:1001B3000075CFC9758400758E0075892075880513
:1001C300758400758A00758B6F758CF4758D6F431C
:1001D300885075840075C90075CA0075CB0075CC4D
:1001E3000075CD0075C80075840175C91875CA807E
:1001F30075CBFB75CDFB75CC80D2CA75840275C9EE
:100203001875CA1275CBF775CDF775CC12D2CA75AE
:10021300840075EF0075A8AF75B80075E6A475E79F
:100223001775F60075F7019000007F007E20E4F05B
:03023300A3DFFC4A
:10023600DEFA7533FF7534FF7535FF7536FF753792
:0E024600FF7538FF7539FF753AFF753BFF22D3
:1030370032C28D32758400C2CF32C0E0C083C082F5
:10304700C0D0C000C0F0C2CFB23720372312250A44
:10305700151BE51B7009751B0A7584017588AF156B
:103067001CE51C7009751C607584027588AF800E9D
:103077001226201529E5297005752904D28B758438
:1030870000D2ECD0F0D000D0D0D082D083D0E032C4
:10309700C2CF32C0E0C0D0E52A6002152AE52D6014
:1030A70002152DE55B6002155B75888FD0D0D0E0E7
:1030B70032C0E0C0D0C084202E1375840F30DF25C6
:1030C700E5E8540FF53CD22E753DC88018153DE54F
:1030D7003D7006E53CD2E7F53C75840F20DF06C25C
:1030E7002ED22DD22920301475840F30F826E5E82A
:1030F70054F0C4F53ED230753FC88018153FE53F00
:103107007006E53ED2E7F53E75840F20F806C2301B
:10311700D22FD228E52B6002152BE55860021558EF
:10312700E55A6002155AE55C6002155CE5626002CB
:103137001562B2A1151DE51D7065751D0AE52C60A8
:1031470002152CE52E6002152EE55D6002155DE582
:103157005E6002155EE55660021556E5576002157A
:0D31670057B2A0E54B6002154BE54C60022D
:10317400154CE54D6002154DE56060021560151EA5
:10318400E51E701E751E0AE55960021559E5616059
:10319400021561151FE51F7009751F06E55F6002C2
:1031A400155FD084C28DD0D0D0E03232202C0DD225
:1031B4002C85BF5585BE5475BB01800BC22C85BFC1
:1031C4005385BE5275BB00C2ED32C0E0C0D0E540AD
:1031D400B4000A054085BE3275BB07803DB4010AC0
:1031E400054085BE2F75BB048030B4020A054085B6
:1031F400BE3275BB068023B4030A054085BE307514
:10320400BB048016B4040A054085BE3275BB058034
:103214000975400085BE3175BB04C2EDD0D0D0E045
:013224003277
:1027870075840FD2FD2275840FC2FD2275840FD286
:10279700FC2275840FC2FC2275840FD2FED21C2244
:1027A70075840FC21CC2FE22C29322D29322758463
:1027B7000FA2FA2275840FA2F92275840FA2DD22D7
:1027C70075840FA2DE22A2922275840FA2DA2275E7
:1027D700840FA2DB2275840FA2D82275840FA2D999
:1027E700220000000000000000000000000000229E
:1027F700C000C001790478B4D8FED9FAD001D0005E
:1028070022C00078141227F7D8FBD00022C0E07549
:102817002A05E52A70FCD0E022C0E0752A0FE52AD8
:1028270070FCD0E022C0E0752A64E52A70FCD0E095
:1028370022A42582F582E58335F0F58322B40A00C8
:1028470022C0E0C3997001D3D0E022B5060122501F
:1028570007B5070122400122D322EF75F0648424D3
:1028670030900061F0E5F0A375F00A842430F0A3FE
:10287700E5F02430F022EF75F06484243090006195
:07288700F0E5F0A375F00A73
:10288E00842430F0A3E5F02430F0900061E0B43001
:10289E000B7420F0A3E0B430037420F02290000EED
:1028AE00E0540FFFA3E0B420028019540FCF75F04F
:1028BE000AA42FFFA3E0B420028009540FCF75F0B5
:1028CE000AA42FFF22C006C005C00490000EE054DB
:1028DE000FFFFEA3E0B42003C3802C540FFDCF7571
:1028EE00F00AA42FFFA3E0B42003C3801A540FFCF8
:1028FE00EE75F064A420D20EFEED75F00AA42E4003
:10290E00052C40028001D3D004D005D0062275F0EC
:10291E006484F6E5F00875F00A84F608A6F008223D
:10292E00C0017900E6B4FF028027F908E6B4FF0380
:10293E00C38022E975F00AA426F908E6B4FF03C3A2
:10294E008013E975F00AA420D207C3264003F9804C
:10295E0004D3D00122E9D00122E675F00AA408269C
:10296E00227843EE12291C7541007542007845907D
:04297E0029C87908E3
:10298200EF134007A3A3A3A3A3801CC0E0C000C011
:1029920001C37905E49336D4A2E4540FF6A318D9FF
:1029A200F3D001D000D0E0D9D8E541600C754209DE
:1029B2007543097544097545098542418543428538
:1029C2004443854544220605020000020105000039
:1029D20004020001000804000200060900040002CB
:0E29E2000901080004080306010806070203A5
:101A760044313233343536373839302A23414243FC
:101A860044AAA3C1C2C3C4D7ABA8A92A23414243CF
:101A96000101010101010101010000000000000037
:101AA6000000000000000000000000000000000030
:101AB6000000000000000000000000000000000020
:101AC6000000000000000000000000000000000010
:101AD6000000000000000000000000000000000000
:101AE60000000000000000000000010101010101EA
:101AF60001010100000000000000000000000000DD
:101B060000000000000000000000000000000000CF
:101B160000000000000000000000000000000000BF
:101B260000000000000000000000000000000000AF
:101B3600000000000000000000000000000000009F
:101B46000000000001010101010101010100000086
:101B5600000000000000000000000000000000007F
:101B6600000000000000000000000000000000006F
:101B7600000000000000000000000000000000005F
:101B8600000000000000000000000000000000004F
:101B9600000000000000000000000000000001013D
:101BA6000101010101010100000000000000000028
:101BB600000000000000000000000000000000001F
:101BC600000000000000000000000000000000000F
:101BD60000000000000000000000000000000000FF
:101BE60000000000000000000000000000000000EF
:101BF60000000000000000000101010101010101D7
:101C060001000000000000000000000000000000CD
:101C160000000000000000000000000000000000BE
:101C260000000000000000000000000000000000AE
:101C3600000000000000000000000000000000009E
:101C4600000000000000000000000000000000008E
:101C56000000010101010101010101000000000075
:101C6600000000000000000000000000000000006E
:101C7600000000000000000000000000000000005E
:101C8600000000000000000000000000000000004E
:101C9600000000000000000000000000000000003E
:101CA60000000000000000000000000020202020AE
:101CB600202020202020202020202020202020201E
:101CC600202020202020202020202020202020200E
:101CD60020202020202020202020202020202020FE
:101CE60020202020202020202020202020202020EE
:101CF60020202020202020202020202020202020DE
:101D060020202020202020202020202020202020CD
:101D160020202020202020202020202020202020BD
:101D260020202020202020202020202020202020AD
:101D3600202020202020202020202020202020209D
:101D4600202020202020202020202020202020208D
:101D5600202020202020202020202020202020207D
:101D6600202020202020202020202020202020206D
:101D7600474C4F42414C20202020202020435443F2
:101D8600535320434F444520202020202020444305
:101D96005320434F44452020202020204C545220DD
:101DA6005245504541544552202020205350454528
:101DB60044204449414C494E472020205350454534
:101DC600442043414C4C494E472020202050544348
:101DD600204E554D424552202020202020564F4966
:101DE6004345204D455353414745532020564F49BF
:101DF600434520504C41594241434B202020494EF7
:101E060056414C49442054595045202020204F55D6
:101E160054204F462052414E4745202020494C4CE5
:101E26004547414C2056414C554520204D5553546D
:101E36002046494C4C204649454C44202020494CDC
:101E46004C4547414C20434F4445202020444154B3
:101E56004120414343455054454420204C494E457A
:101E6600204E554D4245523A20202020555345528A
:101E76002050524F4752414D4D494E4755534552BA
:101E86002049443A2020202020202020564F494334
:101E960045205245434F5244494E472020494C4C19
:101EA6004547414C20454E545259202020494C4C20
:101EB6004547414C2047414E4720202020202043C3
:101EC6004F4D504C45544544202020203633303663
:101ED60037303639343731393734343737303739A4
:101EE600373832353835343838353931353934388C
:101EF60039373431303031303331303731313031B8
:101F060031343131383132333132373133313133A3
:101F16003631343131343631353131353631353982
:101F26003136323136353136373137313137333173
:101F36003737313739313833313836313839313945
:101F46003231393631393932303332303632313056
:101F56003231383232353232393233333234313249
:101F66003530323534303036303037303135303147
:101F76003730323130323330323530323630333139
:101F86003033323033363034333034373035303026
:101F9600353130353330353430363530373130370A
:101FA60032303733303734313134313135313136FF
:101FB60031323231323531333131333231333431FA
:101FC60034313134333134353135323135353135DB
:101FD60036313632313635313732313734323035C3
:101FE60032313232313432323332323532323632C3
:101FF60034333234343234353234363235313235A4
:10200600323235353236313236333236353236368D
:102016003237313237343330363331313331353389
:102026003235333331333332333433333436333575
:10203600313335363336343336353337313431315F
:10204600343132343133343233343331343332345D
:102056003435343436343532343534343535343633
:102066003234363434363534363635303335303628
:102076003531363532333532363533323534363519
:102086003635363036363132363234363237363306
:1020960031363332363534363632363634373033F7
:1020A60037313237323337333137333237333437E8
:1020B60034333735344142434445464748494A4B11
:1020C6004C4D4E4F505152535455565758595A61CC
:1020D60062636465666768696A6B6C6D6E6F707162
:1020E60072737475767778797A303132333435365F
:1020F600373839607E21402324255E262A28295F29
:102106002D2B3D7B7D5B5D7C3A3B3C3E2C2E3F2F51
:1021160020202020202020202064010011022115EB
:102126000101640200110321150101640400110478
:102136002115010164080011052115010178060128
:1021460011060119010182020711072515051982D9
:102156000208110824150A638202091109231500D1
:102166006382020A110A2315006382020B110B24F3
:1021760015006382030C110C261500FF82030D1156
:102186000D261500FF82010E110E27150003820190
:102196000F110F27150003820310111026150AFFD1
:1021A6008203111111261500FF8203121112261542
:1021B60000FF8203131113261500FF820214111467
:1021C60022150063820215111523150063641000A1
:1021D600111621150101642000111728150101822D
:1021E60003161118261500FF644000111901150188
:1021F60001820217111A24150063820218111B248A
:10220600150063820119111C291500026480001152
:102216001D2815010182031A111E261500FF7804D8
:102226001B111F2A17010178041F11202A1701010B
:102236002020202020202020202020202020202098
:102246002020202020202020202020202020202088
:102256002054454C434F2050524F4752414D202069
:1022660020524144494F2050524F4752414D202061
:102276002050484F4E452050524F4752414D202046
:1022860020434F4D50552050524F4752414D20202C
:10229600202041434345535320434F4445202020AB
:1022A6004D4158205245504541542054494D4520F2
:1022B6002056414C4944204D455353414745202023
:1022C600205455524E204F4E2044454C4159202013
:1022D600205455524E204F46462044454C415920E5
:1022E6005455524E2041524F554E4420444C59208D
:1022F60044544D462054454C434F204C4556454C7E
:1023060044544D4620524144494F204C4556454C75
:102316002020564F49434520505245414D502020DC
:1023260020525820505245414D50204741494E2099
:10233600564F49434520584D4954204C4556454C27
:102346002054574F20544F4E45204C4556454C205F
:102356004245455020524144494F204C4556454C34
:10236600424545502054454C434F204C4556454C1C
:10237600434F53204143515549542054494D45201C
:10238600434F532052454C454153452054494D45F2
:10239600494E5445524E414C20535155454C4348A5
:1023A6002020434F5320504F4C415249545920202E
:1023B600434F53205452494747455220564F4C5499
:1023C60054574F20544F4E4520454E41424C4520D0
:1023D60020205245434F52442044454C4159202029
:1023E600202052454144592044454C415920202043
:1023F6004E554D424552204F4620544F4E45532090
:102406002053454E534520504F4C41524954592074
:1024160053454E5345205452494720564F4C54205D
:102426002054574F20544F4E452053454E53452078
:10243600202054574F20544F4E4520434F532020C1
:10244600202020202020202020202020313D454E05
:1024560020202020202020202020202031204D5305
:1024660020202020202020202020203130204D53E5
:1024760020202020202020202020313030204D53C5
:1024860020202020202020202020202020534543CB
:102496002020202020202020202020524154494F57
:1024A60020202020202020202020205441424C455E
:1024B6002020202020202020202020313D504F5356
:1024C6002020202020202020202020204E4D425257
:1024D600202020202020202020202020544F4E4540
:1024E600AF3132333435360A0A0A6314FF3201013A
:1024F600FFFF3232000A8000140180303130323062
:04250600323033003C
:105EBC00755F64E4900000F0301E0B301D24125C02
:105ECC000B122E4080F5301F0B301D16125C4A123F
:105EDC002E4080F530200B301D081233BF122E409F
:035EEC0080F5221C
:102E4000E55F7012900000E0D394004009C21EC2FA
:102E50001FC220C21D22900000E012475F2F5700C2
:102E60002F5A012F5D022F60032F63042F65052F5A
:102E700067062F69072F6C082F6F0A2F720B2F75AB
:102E80000F2F78102F7B142F7E152F81192F841A66
:102E90002F871B2F8A1E2F8D1F2F90232F93242FB8
:102EA00096282F99292F9C2D2F9F2E2FA22F2FA5AB
:102EB000302FA8322FAB332FAD342FB0352FB36462
:102EC0002FB6652FB9662FBC672FBF6E2FC16F2F2E
:102ED000C3703005712FC5782FC7792FC97A300597
:102EE0007B2FCB822FCD832FCF842FD1852FD48CD6
:102EF0002FD78D2FD98E2FDB8F2FDE962FE1972F97
:102F0000E3982FE5992FE8A02FEBA12FEEA22FF049
:102F1000A32FF3AA2FF5AB2FF8AC2FFAAD2FFDB4EA
:102F20003000B53003B63005B73007BE300ABF30C9
:102F30000DC03010C13005C23016F03019F1301C10
:102F4000F2301FFA3022FB3025FC3028FD302BFEFA
:102F5000302EFF0000303102626002616F025B4C74
:102F60000260738004800280000259AC02352D0299
:102F70005F55023AAB0256DF023BF9025734023D7D
:102F800047025B8D02540C02427F025879023E9543
:102F90000258C6023FE3025913024131026018028F
:102FA0005D75025B0A1259F6025527800002506DCA
:102FB000025AC7025789025A3F025DE702558180D3
:102FC000468032804B80408022804580078026806A
:102FD0003F025960024785801C80350257DA024C57
:102FE000B88008802B025BCC0249B7024F8F80204B
:102FF0000248458012024E2C80160237F9024D35E8
:10300000025148800B800C024EA502582A024B1038
:10301000025C8902563302609A0251B102627E025A
:1030200055DB0262F60262F70262F80250DB0262CE
:07303000F9E4900000F0221A
:0F626000E4900002F0755F64900000E004F0220B
:10616F00122ADC122AEB7BFF7A1E7972125F8C7F68
:0F617F0011122AC2C224C221900000E004F022B3
:105B4C0030213D900001E0FFC221BF2A07900000E8
:105B5C00E004F022EF642370277F23122A93900035
:105B6C0002E004F0E0C394034010C21EC21FC22026
:105B7C00C21DE4900000F0025DAE9000007402F0D3
:015B8C0022F6
:106073007BFF7A1E7972125F8C122AEB7F11122A30
:10608300C212628CE490003DF07F2A122A93C2244C
:07609300900000E004F02280
:1059AC00302146900001E0F564C221E564642A6070
:1059BC0038AF6412626F5022AF64122A9390003D8C
:1059CC00E02404F582E43400F583E564F090003DB6
:1059DC00E004F0900000E004F0227BFF7A1E79A234
:0959EC00125F8C90000074FAF0C7
:0159F500228F
:10352D00202103023697900001E0FFC221BF2A0738
:10353D009000007403F022EF6423600302368812BA
:10354D002A93900005E064397077A3E064397071B7
:10355D00A3E06439706BD226900004E0FFB431080B
:10356D00E4900037F00235F7EFB43208E4900038FC
:10357D00F002360AEFB43302803E900004E0FFB44F
:10358D003408E4900039F0023638EFB43508E49091
:10359D00003AF002364EEFB43608E490003BF002EC
:1035AD003664EFB437028010900004E0B438028026
:1035BD0007900004E0B4390B7BFF7A1E79B2023616
:1035CD008EC226900004E0FFB43016A3E0B4301193
:1035DD00A3E0B4300CA3E0B43007900000740AF0FF
:1035ED0022EFB4310C1254CA5007900000740FF042
:1035FD0022900004E0B4320C1253AC50079000003E
:10360D007414F022900004E0B43311A3E0B4300C34
:10361D0012612D50079000007419F022900004E003
:10362D00B4340FA3E0B4300A1261FB900000741E95
:10363D00F022900004E0B4350FA3E0B4300A12621A
:10364D00109000007423F022900004E0B4360FA314
:10365D00E0B4300A1262259000007428F022900028
:10366D0004E0B43716A3E0B43011A3E0B4300CA3DA
:10367D00E0B43007900000742DF0227BFF7A1E79A4
:0A368D00A2125F8C90000074FAF0A6
:013697002210
:105F550090003C740BF090003D7407F0E490004E07
:105F6500F090004FF0900050F07BFF7A1D7972128F
:105F75005F8C125FB77F1E122AC29000007432F048
:015F850022F9
:103AAB00124F1AD3900067E0941F900066E09400C9
:103ABB00400A125F8690000074FAF022900066E0D4
:103ACB00FEA3E0FF90211F75F009124753EE75F02E
:103ADB0009A42583F583E493900045F0902120758C
:103AEB00F009EF124753EE75F009A42583F583E433
:103AFB0093900046F0900066A3E090212175F009A9
:103B0B00124753EE75F009A42583F583E4939000D7
:103B1B0047F090212275F009EF124753EE75F0092B
:103B2B00A42583F583E493900048F0900066A3E00E
:103B3B0090212375F009124753EE75F009A42583E4
:103B4B00F583E493FD900049F090212475F009EF83
:103B5B00124753EE75F009A42583F583E493900087
:103B6B004AF0900066A3E090212575F009124753A7
:103B7B00EE75F009A42583F583E49390004BF09048
:103B8B00212675F009EF124753EE75F009A4258332
:103B9B00F583E49390004CF0900066A3E09021270E
:103BAB0075F009124753EE75F009A42583F583E4EC
:103BBB009390004DF0ED6015900049E075F010A466
:103BCB002436F9742235F0FA7BFF125F8C90004A91
:103BDB00E0FF601175F010A42436F9742235F0FA69
:0E3BEB007BFF125FBD900045E0900000F022CD
:1056DF0090003C7410F090003D7407F090004E74F1
:1056EF0064F090004F740AF0900037E0900050F093
:1056FF007BFF7A1D7982125F8C125FB77F0D122AA2
:10570F00C2900005E0FF122A93900006E0FF122AD4
:10571F0093900007E0FF122A937F1E122AC2900077
:05572F00007432F022BD
:103BF900124F1AD3900067E09400900066E0940099
:103C0900400A125F8690000074FAF022900066E084
:103C1900FEA3E0FF901A9675F009124753EE75F06E
:103C290009A42583F583E493900045F0901A9775CC
:103C3900F009EF124753EE75F009A42583F583E4E3
:103C490093900046F0900066A3E0901A9875F009E9
:103C5900124753EE75F009A42583F583E493900088
:103C690047F0901A9975F009EF124753EE75F0096C
:103C7900A42583F583E493900048F0900066A3E0BF
:103C8900901A9A75F009124753EE75F009A4258325
:103C9900F583E493FD900049F0901A9B75F009EFC4
:103CA900124753EE75F009A42583F583E493900038
:103CB9004AF0900066A3E0901A9C75F009124753E8
:103CC900EE75F009A42583F583E49390004BF090F9
:103CD9001A9D75F009EF124753EE75F009A4258373
:103CE900F583E49390004CF0900066A3E0901A9E4F
:103CF90075F009124753EE75F009A42583F583E49D
:103D09009390004DF0ED6015900049E075F010A416
:103D190024B2F9741C35F0FA7BFF125F8C90004ACB
:103D2900E0FF601175F010A424B2F9741C35F0FAA3
:0E3D39007BFF125FBD900045E0900000F0227D
:1057340090003C7415F090003D7407F090004E7496
:10574400C8F090004F740AF0900038E0900050F0D8
:105754007BFF7A1D7992125F8C125FB77F0C122A3D
:10576400C2900005E0FF122A93900006E0FF122A7F
:1057740093900007E0FF122A937F1E122AC2900022
:05578400007432F02268
:103D4700124F1AD3900067E09400900066E0940049
:103D5700400A125F8690000074FAF022900066E035
:103D6700FEA3E0FF901AF075F009124753EE75F0C5
:103D770009A42583F583E493900045F0901AF17523
:103D8700F009EF124753EE75F009A42583F583E494
:103D970093900046F0900066A3E0901AF275F00940
:103DA700124753EE75F009A42583F583E493900039
:103DB70047F0901AF375F009EF124753EE75F009C3
:103DC700A42583F583E493900048F0900066A3E070
:103DD700901AF475F009124753EE75F009A425837C
:103DE700F583E493FD900049F0901AF575F009EF1B
:103DF700124753EE75F009A42583F583E4939000E9
:103E07004AF0900066A3E0901AF675F0091247533E
:103E1700EE75F009A42583F583E49390004BF090A9
:103E27001AF775F009EF124753EE75F009A42583C9
:103E3700F583E49390004CF0900066A3E0901AF8A5
:103E470075F009124753EE75F009A42583F583E44D
:103E57009390004DF0ED6015900049E075F010A4C7
:103E670024D2F9741C35F0FA7BFF125F8C90004A5C
:103E7700E0FF601175F010A424D2F9741C35F0FA34
:0E3E87007BFF125FBD900045E0900000F0222E
:105B8D007BFF7A1D79A2125F8C7BFF7A1E798212C0
:105B9D005FBD7F0E122AC2900006E0FF122A93907D
:105BAD000007E0FF122A937F1A122AC290003C745C
:0F5BBD001AF090003D7404F09000007432F02252
:10540C003027079000007403F022125FB77F1E1242
:10541C002AC2125219900068E0FEA3E0FFD3940058
:10542C00EE94004030EF94FBEE9400502890003C3A
:10543C00741BF090003D7407F090004E742CF090AB
:10544C00004F740AF0900036E014900050F0900079
:0F545C00007432F022125F8690000074FAF02282
:10427F00D3900067E09400900066E09400400A122B
:10428F005F8690000074FAF022900066E0FEA3E0D3
:10429F00FF901B4A75F009124753EE75F009A425DC
:1042AF0083F583E493900045F0901B4B75F009EF75
:1042BF00124753EE75F009A42583F583E49390001C
:1042CF0046F0900066A3E0901B4C75F0091247531F
:1042DF00EE75F009A42583F583E493900047F090E1
:1042EF001B4D75F009EF124753EE75F009A42583A6
:1042FF00F583E493900048F0900066A3E0901B4E86
:10430F0075F009124753EE75F009A42583F583E480
:10431F0093FD900049F0901B4F75F009EF12475332
:10432F00EE75F009A42583F583E49390004AF0908D
:10433F000066A3E0901B5075F009124753EE75F01D
:10434F0009A42583F583E49390004BF0901B5175DE
:10435F00F009EF124753EE75F009A42583F583E4B6
:10436F009390004CF0900066A3E0901B5275F009FB
:10437F00124753EE75F009A42583F583E49390005B
:10438F004DF0ED6015900049E075F010A424F2F99E
:10439F00741C35F0FA7BFF125F8C90004AE0FF60CF
:1043AF001175F010A424F2F9741C35F0FA7BFF128A
:0B43BF005FBD900045E0900000F02280
:1058790090003C741FF090003D7407F090004E7446
:1058890090F090004F740AF0900039E0900050F0C9
:105899007BFF7A1D79B2125F8C125FB77F0F122AD4
:1058A900C2900006E0FF122A93900007E0FF122A37
:0D58B900937F1E122AC29000007432F0226C
:103E9500124F1AD3900067E09400900066E09400FA
:103EA500400A125F8690000074FAF022900066E0E6
:103EB500FEA3E0FF901BA475F009124753EE75F0C1
:103EC50009A42583F583E493900045F0901BA5751F
:103ED500F009EF124753EE75F009A42583F583E445
:103EE50093900046F0900066A3E0901BA675F0093C
:103EF500124753EE75F009A42583F583E4939000EA
:103F050047F0901BA775F009EF124753EE75F009BE
:103F1500A42583F583E493900048F0900066A3E020
:103F2500901BA875F009124753EE75F009A4258377
:103F3500F583E493FD900049F0901BA975F009EF16
:103F4500124753EE75F009A42583F583E493900099
:103F55004AF0900066A3E0901BAA75F0091247533A
:103F6500EE75F009A42583F583E49390004BF0905A
:103F75001BAB75F009EF124753EE75F009A42583C5
:103F8500F583E49390004CF0900066A3E0901BACA1
:103F950075F009124753EE75F009A42583F583E4FE
:103FA5009390004DF0ED6015900049E075F010A478
:103FB5002412F9741D35F0FA7BFF125F8C90004ACC
:103FC500E0FF601175F010A42412F9741D35F0FAA4
:0E3FD5007BFF125FBD900045E0900000F022DF
:1058C60090003C7424F090003D7407F090004E74F4
:1058D600F4F090004F740AF090003AE0900050F017
:1058E6007BFF7A1D79C2125F8C125FB77F0F122A77
:1058F600C2900006E0FF122A93900007E0FF122AEA
:0D590600937F1E122AC29000007432F0221E
:103FE300124F1AD3900067E09400900066E09400AB
:103FF300400A125F8690000074FAF022900066E097
:10400300FEA3E0FF901BFE75F009124753EE75F017
:1040130009A42583F583E493900045F0901BFF7575
:10402300F009EF124753EE75F009A42583F583E4F5
:1040330093900046F0900066A3E0901C0075F00991
:10404300124753EE75F009A42583F583E49390009A
:1040530047F0901C0175F009EF124753EE75F00914
:10406300A42583F583E493900048F0900066A3E0D1
:10407300901C0275F009124753EE75F009A42583CD
:10408300F583E493FD900049F0901C0375F009EF6C
:10409300124753EE75F009A42583F583E49390004A
:1040A3004AF0900066A3E0901C0475F00912475390
:1040B300EE75F009A42583F583E49390004BF0900B
:1040C3001C0575F009EF124753EE75F009A425831B
:1040D300F583E49390004CF0900066A3E0901C06F7
:1040E30075F009124753EE75F009A42583F583E4AF
:1040F3009390004DF0ED6015900049E075F010A429
:104103002432F9741D35F0FA7BFF125F8C90004A5C
:10411300E0FF601175F010A42432F9741D35F0FA34
:0E4123007BFF125FBD900045E0900000F0228F
:1059130090003C7429F090003D7407F090004E74A1
:1059230058F090004F740AF090003BE0900050F064
:105933007BFF7A1D79D2125F8C125FB77F0D122A1B
:10594300C2900006E0FF122A93900007E0FF122A9C
:0D595300937F1E122AC29000007432F022D1
:10413100124F1AD3900067E09400900066E094005B
:10414100400A125F8690000074FAF022900066E047
:10415100FEA3E0FF901C5875F009124753EE75F06D
:1041610009A42583F583E493900045F0901C5975CB
:10417100F009EF124753EE75F009A42583F583E4A6
:1041810093900046F0900066A3E0901C5A75F009E8
:10419100124753EE75F009A42583F583E49390004B
:1041A10047F0901C5B75F009EF124753EE75F0096B
:1041B100A42583F583E493900048F0900066A3E082
:1041C100901C5C75F009124753EE75F009A4258324
:1041D100F583E493FD900049F0901C5D75F009EFC3
:1041E100124753EE75F009A42583F583E4939000FB
:1041F1004AF0900066A3E0901C5E75F009124753E7
:10420100EE75F009A42583F583E49390004BF090BB
:104211001C5F75F009EF124753EE75F009A4258371
:10422100F583E49390004CF0900066A3E0901C604D
:1042310075F009124753EE75F009A42583F583E45F
:104241009390004DF0ED6015900049E075F010A4D9
:104251002452F9741D35F0FA7BFF125F8C90004AED
:10426100E0FF601175F010A42452F9741D35F0FAC5
:0E4271007BFF125FBD900045E0900000F02240
:106018003020079000007401F02290003C742EF0AC
:1060280090003D7407F07BFF7A1D79E2125F8C12B5
:0E6038005FB77F1E122AC29000007432F02261
:105D7500302707900000742FF02290000BE0643864
:105D85006005A3E0B4390A125F8690000074FAF04A
:105D9500227BFF7A1E7992125F8C90000BE0540FE4
:095DA500F5499000007430F02271
:105B0A0090000BE064386005A3E0B4390A125F869E
:105B1A0090000074FAF0227BFF7A1D79F2125F8CF2
:105B2A0090000BE0540FF549D20AD2127533FF12D6
:105B3A0032257BFF7A1E79C2125F8C90000074FEB8
:025B4A00F02247
:1059F60090000BE0540FF549301E02D208123237E0
:105A0600301E19202F04E52E70F912322E7BFF7AF4
:105A16001E79C2125F8C90000074FEF0301F1920B0
:105A26002D04E52E70F912322E7BFF7A1E79C212F2
:095A36005F8C90000074FEF02268
:10552700302156900001E0FF900035F0C221122A89
:1055370093900035E0FF12626F5021900035E0FF35
:1055470090003DE02404F582E43400F583EFF09009
:10555700003DE004F0900000E004F022900035E008
:10556700B42A079000007403F0227BFF7A1E79A209
:0A557700125F8C90000074FAF0221D
:10506D0030216A900001E0FF900035F0C221122A34
:10507D0093900035E0FFB42A0B90003CE0900000C7
:10508D00F0D22722EFB4230B90003CE0900000F00B
:10509D00C22722900035E0FF12626F50219000353B
:1050AD00E0FF90003DE02404F582E43400F583EF49
:1050BD00F090003DE004F0900000E004F0227BFF52
:0E50CD007A1E79A2125F8C90000074FAF02215
:105AC70030213F900001E0FF900035F0122A93C289
:105AD70021900035E0FFB42A0B90003CE0900000D5
:105AE700F0D22722EFB4230B90003CE0900000F0A7
:105AF700C227227BFF7A1E79A2125F8C9000007466
:035B0700FAF0228F
:0A578900900048E0FF70033027385D
:10579300122AC21260E8124BEA8F64900046E0526C
:1057A30064E56460047F3180027F30122A933027DE
:1057B30017C227E5642430900024F090003474016C
:0857C300F090000074F0F022E8
:0F57CB0090004BE0FF122AC2900000E004F02291
:105A3F00302140900001E0FF900035F0C221122A82
:105A4F0093900035E0FFB42A079000007403F02212
:105A5F0012626F500F900035E090000EF090000032
:105A6F00E004F0227BFF7A1E79A2125F8C90000077
:045A7F0074FAF022A3
:105DE700302132900001E0FF900035F0C221BF2A38
:105DF700079000007403F022900035E0B423079069
:105E07000000E004F0227BFF7A1E79A2125F8C90DB
:065E1700000074FAF02205
:105581001260E890006AEEF0A3EFF0124BEA8F642C
:1055910090003E7401F090000EE0B4310890004696
:1055A100E04264800E90000EE0B4301E900046E0B0
:1055B100F4526490006AE0FEA3E0FFAD64124BADCB
:1055C10012623A90000074FEF0227BFF7A1E79A2EB
:0955D100125F8C90000074FAF0E6
:0155DA0022AE
:104EA500900048E0FF7003302756122AC21260E8CE
:104EB50090006AEEF0A3EFF0E4F564900046E0FFA1
:104EC500E564C39F502790006AE475F00112473DE1
:104ED500AFF0FE124BEA8F6574242564F582E43445
:104EE50000F583E565F0122A93056480CE3027101E
:104EF500C227E56404900034F090000074F0F022BD
:104F050090003D740AF090004BE0FF122AC2900019
:044F150000E004F0C4
:014F19002275
:104E2C00302175900001E0FF900035F0C221122A6C
:104E3C0093900035E0FFB42A079000007403F02231
:104E4C00EFB42308900000E004F0803912626F5038
:104E5C0038900035E0FF90003DE0FE04F074042E25
:104E6C00F582E43400F583EFF0900046E02409FF6E
:104E7C00E433FE90003DE0D39FEE6480F87480989C
:104E8C004016900000E004F0227BFF7A1E79A212FB
:094E9C005F8C90000074FAF02212
:105C8900302137900001E0FF900035F0C221122A3F
:105C990093900035E0FFB42A079000007403F022C6
:105CA900EFB42307900000E004F0227BFF7A1E790D
:0B5CB900A2125F8C90000074FAF02231
:105633001260E890006AEEF0A3EFF090003D740A68
:10564300F0E4F564900046E0FFE564C39F502790C3
:10565300006AE475F00112473DAFF0FE90003DE0B3
:10566300FD04F074042DF582E43400F583E0FD12AB
:105673004BAD056480CE7BFF7A1E79C2125F8C909E
:05568300000074FEF0C0
:0156880022FF
:104F8F0030216B900001E0FF900035F0C221122A12
:104F9F0093900035E0FFB42A079000007403F022CD
:104FAF0012626F501A900035E0FF90003DE0FE0452
:104FBF00F074042EF582E43400F583EFF080107B5B
:104FCF00FF7A1E79A2125F8C90000074FAF0229083
:104FDF000046E02409FFE433FE90003DE0D39FEE4E
:0F4FEF006480F87480984006900000E004F0227F
:10478500900048E0FF7006202703024830122AC235
:104795001260E890006AEEF0A3EFF0124BEA1228DF
:1047A5007D900046E0B40110900063E0FF122A936B
:1047B500900063E0900024F0900046E0B402209061
:1047C5000062E0FF122A93900063E0FF122A9390A3
:1047D5000062E0900024F0900063E0900025F090E6
:1047E5000046E064037030900061E0FF122A939068
:1047F5000062E0FF122A93900063E0FF122A939073
:104805000061E0900024F0900062E0900025F090B7
:104815000063E0900026F0302711C227900046E0A3
:10482500900034F090000074F0F02290004BE0FF0F
:10483500122AC290003D740AF0900000E004F022B4
:105960001228D35002803B1228AB8F6490004CE089
:10597000FFE564C39F402B90004DE0FFE564D39F9B
:1059800050201260E890006AEEF0A3EFF0AD6412D0
:105990004BAD7BFF7A1E79C2125F8C90000074FEC3
:0B59A000F022125F8690000074FAF005
:0159AB0022D9
:1057DA001228D35002803F1228AB8F6490004CE00D
:1057EA00FFE564C39F400B90004DE0FFE564D39F43
:1057FA004004E56470201260E890006AEEF0A3EFBE
:10580A00F0AD64124BAD7BFF7A1E79C2125F8C90A9
:0F581A00000074FEF022125F8690000074FAF016
:01582900225C
:104CB800900048E0FF700330275E122AC21260E8B5
:104CC80090006AEEF0A3EFF0124BEA8F64124C33B7
:104CD800E4F56474612564F582E43400F583E0FF4B
:104CE80074242564F582E43400F583EFF0746125BB
:104CF80064F582E43400F583E0FF122A930564E545
:104D080064C3940440CD30270FC227900034740345
:104D1800F090000074F0F02290004BE0FF122AC2DD
:0C4D280090003D740AF0900000E004F0E0
:014D3400225C
:105BCC007F0A1244D28F64E56460121260E8900080
:105BDC006AEEF0A3EFF0E56414FD124BADE5647BC7
:105BEC00FF600E7A1E79C2125F8C90000074FEF07A
:0E5BFC00227A1E7942125F8C90000074FAF03B
:015C0A002277
:1049B700900048E0FF7006202703024A52122AC2DD
:1049C7001260E890006AEEF0A3EFF0124BEA1228AB
:1049D7007D90006AE475F00112473DAFF0FE124B7F
:1049E700EA122861900062E0FF900024F0A3F01221
:1049F7002A93900063E0FF122A9390006AE475F00F
:104A07000112473DAFF0FE124BEA12286190006198
:104A1700E0FF900026F0900062E0900027F0900001
:104A270063E0900028F0122A93900062E0FF122AB8
:104A370093900063E0FF122A9330270FC22790005C
:104A4700347405F090000074F0F02290004BE0FF02
:104A5700122AC290003D740AF0900000E004F02290
:1048450090000EE0540F75F00AA4FFA3E0540F2F5B
:10485500F564900011E0540F75F00AA4FDACF090DA
:104865000010E0540F75F064A42DFFE5F03CFE90B8
:104875000012E0540F7C002FFFEC3EFEE564C3946C
:10488500014019E564D394145012C3EF9401EE94DA
:10489500004009D3EF94FAEE9400400A125F869027
:1048A500000074FAF0221260E890006AEEF0A3EFBF
:1048B500F090006AE475F00112473DAFF0FEAD647B
:1048C500124BAD900011E0540F75F00AA4FF900053
:1048D50010E0540F75F064A42FFF900012E0540F00
:1048E5002FF56490006AE0FEA3E0FFAD64124BADC6
:0F48F5007BFF7A1E79C2125F8C90000074FEF078
:014904002290
:1037F9007F0D1244D2EF701A900011E0B43010A37B
:10380900E0B4300BA3E0B43006A3E06430600302F7
:1038190038F2900015E0FF64306004EFB4350E9083
:103829000016E0540FD3940540030238F2900015B6
:10383900E0FF64316004EFB4361190001AE0B4205F
:1038490007900019E0B420030238F2900015E0FF58
:1038590064326004EFB43711900019E0B420079086
:103869000018E0B420030238F2900015E0FF643339
:103879006004EFB43809900016E0B42002806A9021
:103889000015E0FF64346005EF6439706690001636
:10389900E0540F75F00AA4FFA3E0540F2FF56490CC
:1038A9000019E0540F75F00AA4FDACF0900018E07F
:1038B900540F75F064A42DFFE5F03CFE90001AE06A
:1038C900540F7C002FFFEC3EFEE564C394014019C0
:1038D900E564D394145012C3EF9401EE94004009A7
:1038E900D3EF94FAEE9400400A125F8690000074B8
:1038F900FAF0221260E890006AEEF0A3EFF090006F
:103909003D740AF0E4F564900046E0FFE564C39F66
:10391900502790006AE475F00112473DAFF0FE9020
:10392900003DE0FD04F074042DF582E43400F583D4
:10393900E0FD124BAD056480CE7BFF7A1E79C21281
:083949005F8C90000074FEF099
:013951002253
:104D3500900048E0FF700330275B122AC21260E83A
:104D450090006AEEF0A3EFF0E4F564900046E0FF12
:104D5500E564C39F502C90006AE475F00112473D4D
:104D6500AFF0FE124BEA8F6574242564F582E434B6
:104D750000F583E565F07E00124BEA122A9305647F
:104D850080C9302710C227E56404900034F09000F4
:104D95000074F0F02290004BE0FF122AC290003D13
:0B4DA500740AF0D224900000E004F03B
:014DB00022E0
:10514800302165900001E0FF900035F0C221BF2AB0
:10515800079000007403F022900035E0FFB42308A4
:10516800900000E004F0803DEF547FFF122A9390F6
:105178000035E0547FFF90003DE0FE04F074042EFB
:10518800F582E43400F583EFF0900046E02409FF4F
:10519800E433FE90003DE0D39FEE6480F87480987D
:0951A8004006900000E004F02232
:10582A0030214B900001E0FF900035F0C221BF2AE1
:10583A00079000007403F022900035E0FFB4230BB8
:10584A00900000E004F0E004F0801012626F500F44
:10585A00900035E0900040F0900000E004F0227BD8
:0F586A00FF7A1E79A2125F8C90000074FAF02270
:104B1000202103024BAC900001E0FF900035F0C271
:104B200021BF2A079000007403F022900035E0FFB7
:104B3000B4230A900000E004F0E004F02212626F57
:104B4000505B900040E0540F75F00AA4FF900035D0
:104B5000E0540F2FF0E09020BB93FF900035F0124F
:104B60002A93900035E0FF90003DE0FE04F07404CD
:104B70002EF582E43400F583EFF0900046E024093E
:104B8000FFE433FE90003DE0D39FEE6480F8748034
:104B900098900000E0400304F02214F0227BFF7A9A
:0D4BA0001E79A2125F8C90000074FAF022C2
:10609A00301E09900077E0F55E122787302003E46E
:1060AA00F55E301F0B301C05755E0A8003755E288D
:0760BA00900000E004F02259
:1051B100E55E70631245C0900045E012475F51E122
:1051C1006451E66E51E67851E68251E68C51EB96D8
:1051D10051F0A051F5AA51FAB451FFBE000052029C
:1051E1001261E4801C125FE880171262FA801212C9
:1051F10062FB800D1262FC80081262FD8003126264
:10520100FE301E0D900076E0F55A900000E004F0AB
:08521100229000007401F0225C
:0E627E00E55A700912278D9000007401F0227D
:1055DB00301E0D900077E0F55E122787E55E70FCBC
:1055EB00301F07755E05E55E70FCE4F564301F0C3B
:1055FB001262BC12282C1262E212282C301E0C12E2
:10560B0062C712282C1262E212282C0564E564C3CF
:10561B00940540D9301E0A900076E0F55AE55A7091
:07562B00FC9000007401F087
:015632002255
:0162F6002285
:0162F7002284
:0162F8002283
:1050DB00301F0A201C079000007401F022301E0DB7
:1050EB00900077E0F55E122787E55E70FC301F07B6
:1050FB00755E05E55E70FC301E151262C7E4F56443
:10510B0012282C0564E564C3940A40F41262E23061
:10511B001F151262BCE4F56412282C0564E564C308
:10512B00940A40F41262E2301E0A900076E0F55ABF
:0C513B00E55A70FC125DAEE4900000F03C
:015147002245
:0162F9002282
:105C0B00302F3B202138755F64E53E547FFF901A9F
:105C1B007693900001F030240EE53E30E709EF90CB
:105C2B001A8693900001F0D221C22F900001E0B4AC
:0F5C3B002307900002E004F022E4900002F02220
:105C4A00302D3B202138755F64E53C547FFF901A64
:105C5A007693900001F030240EE53C30E709EF908E
:105C6A001A8693900001F0D221C22D900001E0B46F
:0F5C7A002307900002E004F022E4900002F022E1
:1033BF0020220302352C30210302352C900002E02D
:1033CF00F564E4F0755F641262F0D221BF300790AC
:1033DF0000017430F022BF31079000017431F022E8
:1033EF00BF32079000017432F022BF330790000103
:1033FF007433F022BF34079000017434F022BF35CC
:10340F00079000017435F022BF3607900001743623
:10341F00F022BF37079000017437F022BF380790B2
:10342F0000017438F022BF39079000017439F0227F
:10343F00BF23109000017423F0AF64056490000265
:10344F00EFF022BF2A07900001742AF022BF410734
:10345F009000017441F022BF42079000017442F0C6
:10346F0022BF43079000017443F022BF640790000E
:10347F00017444F022202403C22122BF610790006F
:10348F00017461F022BF62079000017462F022BFE5
:10349F0063079000017463F022BF6407900001740A
:1034AF0064F022BF65079000017465F022BF6607C4
:1034BF009000017466F022BF67079000017467F0F7
:1034CF0022BF68079000017468F022BF690790005F
:1034DF00017469F022BF6A07900001746AF022BF7D
:1034EF006B07900001746BF022BF6C0790000174A2
:1034FF006CF022BF6D07900001746DF022BF6E0754
:10350F00900001746EF022BF6F07900001746FF08E
:0D351F0022BF70079000017470F022C221DD
:01352C00227C
:0B628C007F209000047420F0A3DFFCD2
:0162970022E4
:0F626F00EFC394304007EFD39439500122C3227C
:104F1A0090000DE0FD6420602E90000CE0540F75A7
:104F2A00F00AA4FBAAF090000BE0540F75F064A4F9
:104F3A002BFFE5F03AFEED540F7C002FFFEC3E907C
:104F4A000066F0A3EF803190000CE0FD6420900031
:104F5A000B601AE0540F75F00AA4FFED540F7C00A1
:104F6A002FFEEC35F0900066F0A3CE800BE0540FD4
:104F7A00FF900066E4F0A3EFF0E024FFF0900066F3
:054F8A00E034FFF022FD
:1052190090000AE0FD6420602B900009E0540F75AE
:10522900F00AA4FBAAF0900008E0540F75F064A4FA
:105239002BFFE5F03AFEED540F7C002FFFEC3E907A
:105249000068802E900009E0FD6420900008601A33
:10525900E0540F75F00AA4FFED540F7C002FFEEC0B
:1052690035F0900068F0A3CEF022E0540FFF9000D3
:0752790068E4F0A3EFF0224E
:10612D00900006E0540F75F00AA4FFA3E0540F2F62
:10613D00900036F0D394004006E09415500122C330
:01614D00222F
:1054CA00E4FFEF75F003A424D2F582E4341EF583D9
:1054DA00E493FE900005E0FDEE6D703BEF75F0037E
:1054EA00A424D3F582E4341EF583E493FE900006E7
:1054FA00E0FDEEB50521EF75F003A424D4F582E4AE
:10550A00341EF583E493FE900007E0FDEEB505072F
:0C551A00900037EFF0D3220FBF33A7C37F
:015526002262
:1053AC00E4FF75F003EFA4246BF582E5F0341FF5F0
:1053BC0083E493FE900005E0FDEE6D703D75F00307
:1053CC00EFA4246CF582E5F0341FF583E493FE9092
:1053DC000006E0FDEEB5052275F003EFA4246DF593
:1053EC0082E5F0341FF583E493FE900007E0FDEEB8
:0F53FC00B50507900038EFF0D3220FBF70A4C3A0
:01540B00227E
:1044D20074042FF582E43400F583E0FD64317069E1
:1044E200FE74052FF582E43400F583E0FCEE75F0EE
:1044F20003A424D2F582E4341EF583E4936C704263
:1045020074062FF582E43400F583E0FCEE75F003C7
:10451200A424D3F582E4341EF583E493B504237412
:10452200072FF582E43400F583E0FCEE75F003A476
:1045320024D4F582E4341EF583E493B50404EE0436
:10454200FF220EBE339B7F0022ED6432706DFE743B
:10455200052FF582E43400F583E0FD75F003EEA447
:10456200246BF582E5F0341FF583E4936D70457496
:10457200062FF582E43400F583E0FD75F003EEA426
:10458200246CF582E5F0341FF583E493B5052574B8
:10459200072FF582E43400F583E0FD75F003EEA405
:1045A200246DF582E5F0341FF583E493B50505EE3D
:0D45B2002434FF220EBE70977F00227F0090
:0145BF0022D9
:104C3300EFC3943390006150397431F0EF75F00392
:104C4300A424D2F582E4341EF583E493900062F049
:104C5300EF75F003A424D3F582E4341EF583E493C3
:104C6300900063F0EF75F003A424D4F582E4341EBE
:104C7300803A7432F075F003EFA424D2F582E5F0A4
:104C8300341EF583E493900062F075F003EFA424DF
:104C9300D3F582E5F0341EF583E493900063F07559
:104CA300F003EFA424D4F582E5F0341EF583E493F6
:054CB300900064F022F6
:1061FB00900006E0540F75F00AA4FFA3E0540F2F94
:05620B00900039F022B3
:10621000900006E0540F75F00AA4FFA3E0540F2F7E
:0562200090003AF0229D
:10622500900006E0540F75F00AA4FFA3E0540F2F69
:0562350090003BF02287
:065F86007BFF7A1E791278
:065F8C008B688A69896A36
:105F92007F01122AC2E4F56BAB68AA69A96A856B14
:105FA200827583001246A9FF122A93056BE56BC323
:045FB200941040E423
:015FB60022C8
:065FB7007BFF7A1E7962F7
:065FBD008B688A69896A05
:105FC3007F11122AC2E4F56BAB68AA69A96A856BD3
:105FD300827583001246A9FF122A93056BE56BC3F2
:045FE300941040E4F2
:015FE7002297
:1060E800900050E0FF90004FE08FF0A4FF90004E2A
:1060F800E07C002FFFEC35F0FE900047E02FFFEC2E
:036108003EFE2236
:10623A00900049E075F010A42436F9742235F0FA7A
:05624A007BFF025FBDB7
:0362F0007F032207
:1061C900E4F564AF647E00E5649024E693FD124B28
:0A61D900AD0564E564C3942340E9BA
:0161E3002299
:1060C100E4F564AF647E00124BEA746C2564F582DA
:1060D100E43400F583EFF00564E564C3942340E301
:0660E10090006CE0F520C8
:0160E7002296
:1061E400301E08900024E0FF1262A4301F089000C3
:0761F40024E0FF1262982273
:105FE800E4F564900034E0FFE564C39F5021742415
:105FF8002564F582E43400F583E0F565301E04FF7E
:0F6008001262A4301F05AF65126298056480D440
:016017002266
:0162FA002281
:0162FB002280
:0162FC00227F
:0162FD00227E
:0162FE00227D
:0C6298001262D212282C1262E902282C9B
:0C62A4001262DA12282C1262E902282C87
:1045C000E4F564F565F566900067E02401FF90006E
:1045D00066E03400FEC3EF940AEE94005005A3E0B9
:1045E00004F566D3EF9463EE9400404C900067E0CE
:1045F0002401FB900066E03400FA7C007D64AF0388
:10460000FE1246E88F64EF75F064A4FFC3EB9FFFD2
:10461000EA95F0FE7C007D0A1246E88F65A3E0046F
:10462000FFE56475F064A4FEC3EF9EFFE56575F0D9
:104630000AA4FEC3EF9EF566900067E02401FF9098
:104640000066E03400FED3EF9409EE940040197C3C
:10465000007D0A1246E88F65A3E004FFE56575F06A
:104660000AA4FEC3EF9EF56674302564F5647430C9
:104670002565F56574302566F566301E14AF641245
:1046800062A4AF651262A4AF661262A47F2A1262AE
:10469000A4301F14AF64126298AF65126298AF66BF
:0846A0001262987F2A12629851
:0146A80022EF
:1032250075480012324050FB227548001232C950D1
:10323500FB2275480012328050FB22758400E54858
:1032450075F003A490324D730232E50232F4023375
:10325500120232FB02331E02332502332D0232F4F1
:1032650002333B0232FB02334B0233540232E50296
:1032750032F40233620232FB02336E758400E54894
:1032850075F003A490328D730232E50232F40233F5
:10329500120232FB02331E0233250232E50232F4FA
:1032A5000233120232FB02331E02332502331E02A1
:1032B500332502332D0232F40233700232FB02331E
:1032C5004B02336E758400E54875F003A49032D641
:1032D500730232E50232F40233620232FB02336ECC
:1032E500C2FA123380123380759B000548C3223021
:1032F500F9020548C32230F912E59A20E7FB12339B
:1033050080D2FA1233801233800548C322C2FA12E2
:103315003380759B040548C322752D1E0548C322BD
:10332500E52D70020548C322C2FA1233801233A17B
:10333500F59B0548C322C2FA1233801233B0440705
:10334500F59B0548C322123392F52E0548C3227515
:10335500840F30DE04E52E70020548C322C2FA123E
:103365003380759B080548C322D322C2FA123380E5
:093375001233B04405F59B054834
:10337E00C32200000000000000000000000000005A
:10338E0000000022903399E54993225A5A5A5A5A0C
:10339E00FAFAFA9033A8E549932200B45AE12D8740
:1033AE007ADB9033B7E549932200000000000080DD
:0133BE00808E
:10546B0075840F1200A41260C1126046125DAE1259
:10547B00614E125689125280302B05124DB1C22B40
:10548B00302A28C22A7F0C122B091261C91260C163
:10549B00126046C21EC21FC220E4F56312282C05FF
:1054AB0063E563C3941E40F4125DAE301DC4125EFF
:0F54BB00BC1260C1126046C21EC21FC22080B365
:10528000900041E070141227D0400F12279F7562E2
:10529000641262BC900041E004F0900041E0B4016F
:1052A00010E562703E1262E275613C900041E004DC
:1052B000F0900041E06402701E1227E250051227B0
:1052C000DC4007E5617010201D0D1227A775626490
:1052D000900041E004F022900041E0B40305E56253
:0452E0007001F02247
:1043CA0009920A9E0BC70D100E7D101211D213C549
:1043DA0015ED185208D0094E09D40A600AF40B9157
:1043EA000C360CE50D9D0E600F2D100610EB11DD3D
:1043FA0012DC13EA15071633177118C01D2107B10D
:10440A0007E808200859196E1A211ADA1B971C5A4C
:10441A000894090E09900A190AA90B410BE30C8C9E
:10442A000D3F0DFD0EC50F9810771162125B1362D6
:10443A001477159B16D018161DEF1EC21F9B2079E4
:10444A00215F224A233B24342533263912330FCDE8
:10445A0014331566169A17CD19000E9A13661100B1
:10446A0011661033150016331766189A19CD0DCD3B
:10447A000F00129A11CD1300149A15CD1700183394
:10448A0019660E330F66109A191823A01296203D4A
:10449A00129623A0129627631488203D148823A01D
:1044AA001488276316B8203D16B823A016B82763C8
:1044BA001918203D1918276312962B8C14882B8CF7
:0844CA0016B82B8C19182B8C7D
:10395200900043E0FF705930181C90008BE0540F28
:1039620075F014A424CAF582E43443F583C083C0FD
:103972008290008C801A900087E0540F75F014A496
:1039820024CAF582E43443F583C083C08290008860
:10399200E0540FD082D08375F002124753E493F5BE
:1039A20008740193F509D231D21375600A023A9173
:1039B200EF64016003023A99E5606002C322756018
:1039C2001E30186690008DE0540F75F014A424CABE
:1039D200F582E43443F583C083C08290008EE054C4
:1039E2000FD082D08375F002124753E493F5087426
:1039F2000193F50990008BE0540F75F014A424CACA
:103A0200F582E43443F583C083C08290008CE05495
:103A12000FD082D08375F002124753740193650967
:103A22007004E493650870678062900089E0540F27
:103A320075F014A424CAF582E43443F583C083C02C
:103A42008290008AE0540FD082D08375F002124730
:103A520053E493F508740193F509900087E0540F3D
:103A620075F014A424CAF582E43443F583C083C0FC
:103A720082900088E0540FD082D08375F002124702
:103A820053740193B50908E493B508037560469031
:103A92000043E004F0C322900043E0B4020AE56070
:093AA2006002C3221262E2D32289
:0B62BC0075081575095ED231D20B2267
:0B62C70075081575095ED231D2132254
:0762E200C231C20BC21322FE
:0862D200123698D232D20C22E0
:0862DA00123698D232D21422D0
:09369800E4F512F513F514F51523
:1036A100EF12475F379C23378B2A36D93036EB31FF
:1036B10036FD32370F333721343733353745363717
:1036C1005737376938377A3937AD4137BE4237CF47
:1036D1004337E044000037F8904492E493F50D74C9
:1036E1000193F50E9044940237EF904496E493F5DC
:1036F1000D740193F50E9044980237EF90449AE4CB
:1037010093F50D740193F50E90449C0237EF9044AC
:103711009EE493F50D740193F50E9044A00237EFEA
:103721009044A2E493F50D740193F50E9044A40224
:1037310037EF9044A6E493F50D740193F50E904490
:10374100A80237EF9044AAE493F50D740193F50EA6
:103751009044AC0237EF9044AEE493F50D740193BD
:10376100F50E9044B00237EF9044B2E493F50D7436
:103771000193F50E9044B480759044B6E493F50D31
:10378100740193F50E9044B880649044BAE493F5C3
:103791000D740193F50E9044BC80539044BEE493A4
:1037A100F50D740193F50E9044C080429044C2E43B
:1037B10093F50D740193F50E9044C480319044C685
:1037C100E493F50D740193F50E9044C88020904464
:1037D100CAE493F50D740193F50E9044CC800F90DB
:1037E10044CEE493F50D740193F50E9044D0E49327
:0837F100F50F740193F510229D
:0762E900C232C214C20C22F4
:1002540020202020202053494E4520574156452038
:1002640000465245513A2020313030302020204879
:100274007A000007000E0014001B00220029003041
:100284000037003D0044004B0052005900600066F6
:10029400006D0074007B00820089008F0096009D31
:1002A40000A400AB00B100B800BF00C600CD00D46C
:1002B40000DA00E100E800EF00F600FD0103010AA6
:1002C40001110118011F0126012C0133013A0141DA
:1002D4000148014F0155015C0163016A0171017715
:1002E400017E0185018C0193019A01A001A701AE51
:1002F40001B501BC01C301C901D001D701DE01E58B
:1003040001EC01F201F902000207020E0214021BC1
:100314000222022902300237023D0244024B0252F9
:10032400025902600266026D0274027B0282028933
:10033400028F0296029D02A402AB02B102B802BF70
:1003440002C602CD02D402DA02E102E802EF02F6AA
:1003540002FD0303030A03110318031F0326032CDE
:100364000333033A03410348034E0355035C036319
:10037400036A03710377037E0385038C0393039A53
:1003840003A003A703AE03B503BC03C303C903D08F
:1003940003D703DE03E503EC03F203F904000407C7
:1003A400040E0414041B0422042904300437043DFD
:1003B4000444044B0452045904600466046D047438
:1003C400047B04820489048F0496049D04A404AB72
:1003D40004B104B804BF04C604CD04D404DA04E1AF
:1003E40004E804EF04F604FD0503050A05110518E5
:1003F400051F0526052C0533053A05410548054E1C
:100404000555055C0563056A05710577057E058557
:10041400058C0593059A05A005A705AE05B505BC91
:1004240005C305C905D005D705DE05E505EB05F2CD
:1004340005F906000607060E0614061B0622062901
:1004440006300637063D0644064B0652065906603A
:100454000666066D0674067B06820689068F069676
:10046400069D06A406AB06B106B806BF06C606CDB1
:1004740006D406DA06E106E806EF06F606FD0703EB
:10048400070A07110718071F0726072C0733073A1F
:1004940007410748074E0755075C0763076A07715A
:1004A4000777077E0785078C0793079A07A007A796
:1004B40007AE07B507BC07C307C907D007D707DED0
:1004C40007E507EB07F207F908000807080E081408
:1004D400081B0822082908300837083D0844084B3F
:1004E4000852085908600866086D0874087B088279
:1004F4000889088F0896089D08A408AB08B108B8B5
:1005040008BF08C608CD08D408DA08E108E808EFEF
:1005140008F608FD0903090A09110918091F092623
:10052400092C0933093A09410948094E0955095C5E
:100534000963096A09710977097E0985098C099398
:10054400099A09A009A709AE09B509BC09C309C9D3
:1005540009D009D709DE09E509EB09F209F90A000E
:100564000A070A0E0A140A1B0A220A290A300A3741
:100574000A3D0A440A4B0A520A590A600A660A6D7D
:100584000A740A7B0A820A880A8F0A960A9D0AA4B8
:100594000AAB0AB10AB80ABF0AC60ACD0AD40ADAF3
:1005A4000AE10AE80AEF0AF60AFD0B030B0A0B112B
:1005B4000B180B1F0B260B2C0B330B3A0B410B4860
:1005C4000B4E0B550B5C0B630B6A0B710B770B7E9D
:1005D4000B850B8C0B930B9A0BA00BA70BAE0BB5D7
:1005E4000BBC0BC30BC90BD00BD70BDE0BE50BEB12
:1005F4000BF20BF90C000C070C0E0C140C1B0C2248
:100604000C290C300C370C3D0C440C4B0C520C597F
:100614000C600C660C6D0C740C7B0C820C880C8FBB
:100624000C960C9D0CA40CAB0CB10CB80CBF0CC6F6
:100634000CCD0CD40CDA0CE10CE80CEF0CF60CFD30
:100644000D030D0A0D110D180D1F0D250D2C0D3365
:100654000D3A0D410D480D4E0D550D5C0D630D6A9F
:100664000D710D770D7E0D850D8C0D930D9A0DA0DA
:100674000DA70DAE0DB50DBC0DC30DC90DD00DD715
:100684000DDE0DE50DEB0DF20DF90E000E070E0E4D
:100694000E140E1B0E220E290E300E370E3D0E4484
:1006A4000E4B0E520E590E600E660E6D0E740E7BBE
:1006B4000E820E880E8F0E960E9D0EA40EAB0EB1FA
:1006C4000EB80EBF0EC60ECD0ED40EDA0EE10EE835
:1006D4000EEF0EF60EFD0F030F0A0F110F180F1F6A
:1006E4000F250F2C0F330F3A0F410F480F4E0F55A4
:1006F4000F5C0F630F6A0F710F770F7E0F850F8CDE
:100704000F930F9A0FA00FA70FAE0FB50FBC0FC218
:100714000FC90FD00FD70FDE0FE50FEB0FF20FF954
:1007240010001007100E1014101B10221029103086
:100734001037103D1044104B1052105910601066C1
:10074400106D1074107B10821088108F1096109DFD
:1007540010A410AB10B110B810BF10C610CD10D437
:1007640010DA10E110E810EF10F610FD1103110A71
:1007740011111118111F1125112C1133113A1141A6
:100784001148114E1155115C1163116A11711177E1
:10079400117E1185118C1193119A11A011A711AE1C
:1007A40011B511BC11C211C911D011D711DE11E557
:1007B40011EB11F211F912001207120E1214121B8E
:1007C4001222122912301237123D1244124B1252C5
:1007D400125912601266126D1274127B1282128800
:1007E400128F1296129D12A412AB12B112B812BF3C
:1007F40012C612CD12D412DA12E112E812EF12F676
:1008040012FD1303130A13111318131F1325132CAA
:100814001333133A13411348134E1355135C1363E4
:10082400136A13711377137E1385138C1393139A1E
:1008340013A013A713AE13B513BC13C213C913D05B
:1008440013D713DE13E513EB13F213F91400140793
:10085400140E1414141B1422142914301437143DC8
:100864001444144B14521459145F1466146D147404
:10087400147B14821488148F1496149D14A414AB3E
:1008840014B114B814BF14C614CD14D414DA14E17A
:1008940014E814EF14F614FD1503150A15111518B0
:1008A400151F1525152C1533153A15411548154EE8
:1008B4001555155C1563156A15711577157E158523
:1008C400158C1593159A15A015A715AE15B515BC5D
:1008D40015C215C915D015D715DE15E515EB15F29A
:1008E40015F916001607160E1614161B16221629CD
:1008F40016301637163D1644164B16521659165F07
:100904001666166D1674167B16821688168F169642
:10091400169D16A416AB16B116B816BF16C616CD7C
:1009240016D416DA16E116E816EF16F616FC1703B7
:10093400170A17111718171F1725172C1733173AEB
:1009440017411748174E1755175C1763176A177125
:100954001777177E1785178C1793179A17A017A761
:1009640017AE17B517BC17C217C917D017D717DE9C
:1009740017E517EB17F217F918001807180E1814D3
:10098400181B1822182918301837183D1844184B0A
:1009940018521859185F1866186D1874187B188245
:1009A4001888188F1896189D18A418AB18B118B881
:1009B40018BF18C618CD18D418DA18E118E818EFBB
:1009C40018F618FC1903190A19111918191F1925F1
:1009D400192C1933193A19411948194E1955195C2A
:1009E4001963196A19711977197E1985198C199364
:1009F400199A19A019A719AE19B519BC19C219C9A0
:100A040019D019D719DE19E519EB19F219F91A00D9
:100A14001A071A0E1A141A1B1A221A291A301A370C
:100A24001A3D1A441A4B1A521A591A5F1A661A6D49
:100A34001A741A7B1A821A881A8F1A961A9D1AA483
:100A44001AAB1AB11AB81ABF1AC61ACD1AD41ADABE
:100A54001AE11AE81AEF1AF61AFC1B031B0A1B11F7
:100A64001B181B1F1B251B2C1B331B3A1B411B482C
:100A74001B4E1B551B5C1B631B6A1B711B771B7E68
:100A84001B851B8C1B931B991BA01BA71BAE1BB5A3
:100A94001BBC1BC21BC91BD01BD71BDE1BE51BEBDE
:100AA4001BF21BF91C001C071C0E1C141C1B1C2213
:100AB4001C291C301C371C3D1C441C4B1C521C594B
:100AC4001C5F1C661C6D1C741C7B1C821C881C8F88
:100AD4001C961C9D1CA41CAB1CB11CB81CBF1CC6C2
:100AE4001CCD1CD41CDA1CE11CE81CEF1CF61CFCFD
:100AF4001D031D0A1D111D181D1F1D251D2C1D3331
:100B04001D3A1D411D481D4E1D551D5C1D631D6A6A
:100B14001D711D771D7E1D851D8C1D931D991DA0A6
:100B24001DA71DAE1DB51DBC1DC21DC91DD01DD7E1
:100B34001DDE1DE51DEB1DF21DF91E001E071E0E18
:100B44001E141E1B1E221E291E301E361E3D1E4450
:100B54001E4B1E521E591E5F1E661E6D1E741E7B8A
:100B64001E821E881E8F1E961E9D1EA41EAB1EB1C5
:100B74001EB81EBF1EC61ECD1ED41EDA1EE11EE800
:100B84001EEF1EF61EFC1F031F0A1F111F181F1F36
:100B94001F251F2C1F331F3A1F411F481F4E1F556F
:100BA4001F5C1F631F6A1F711F771F7E1F851F8CA9
:100BB4001F931F991FA01FA71FAE1FB51FBC1FC2E5
:100BC4001FC91FD01FD71FDE1FE51FEB1FF21FF920
:100BD40020002007200E2014201B20222029203052
:100BE4002036203D2044204B20522059205F20668F
:100BF400206D2074207B20822088208F2096209DC9
:100C040020A420AB20B120B820BF20C620CD20D303
:100C140020DA20E120E820EF20F620FC2103210A3D
:100C240021112118211F2125212C2133213A214171
:100C34002148214E2155215C2163216A21712177AC
:100C4400217E2185218C2193219921A021A721AEE8
:100C540021B521BC21C221C921D021D721DE21E522
:100C640021EB21F221F922002207220E2214221B59
:100C74002222222922302236223D2244224B225291
:100C84002259225F2266226D2274227B22822288CC
:100C9400228F2296229D22A422AB22B122B822BF07
:100CA40022C622CD22D322DA22E122E822EF22F642
:100CB40022FC2303230A23112318231F2325232C77
:100CC4002333233A23412348234E2355235C2363B0
:100CD400236A23712377237E2385238C23932399EB
:100CE40023A023A723AE23B523BC23C223C923D027
:100CF40023D723DE23E523EB23F223F9240024075F
:100D0400240E2414241B2422242924302436243D94
:100D14002444244B24522459245F2466246D2474CF
:100D2400247B24822488248F2496249D24A424AB09
:100D340024B124B824BF24C624CD24D324DA24E146
:100D440024E824EF24F624FC2503250A251125187C
:100D5400251F2525252C2533253A25412548254EB3
:100D64002555255C2563256A25702577257E2585EF
:100D7400258C2593259925A025A725AE25B525BC29
:100D840025C225C925D025D725DE25E525EB25F265
:100D940025F926002607260E2614261B2622262998
:100DA40026302636263D2644264B26522659265FD3
:100DB4002666266D2674267B26822688268F26960E
:100DC400269D26A426AB26B126B826BF26C626CD48
:100DD40026D326DA26E126E826EF26F626FC270384
:100DE400270A27112718271F2725272C2733273AB7
:100DF40027412748274E2755275C2763276A2770F2
:100E04002777277E2785278C2793279927A027A72D
:100E140027AE27B527BC27C227C927D027D727DE67
:100E240027E527EB27F227F928002807280D28149F
:100E3400281B2822282928302836283D2844284BD6
:100E440028522859285F2866286D2874287B288210
:100E54002888288F2896289D28A428AB28B128B84C
:100E640028BF28C628CD28D328DA28E128E828EF87
:100E740028F628FC2903290A29112918291F2925BC
:100E8400292C2933293A29412948294E2955295CF5
:100E94002963296A29702977297E2985298C299330
:100EA400299929A029A729AE29B529BC29C229C96C
:100EB40029D029D729DE29E529EB29F229F92A00A5
:100EC4002A072A0D2A142A1B2A222A292A302A36DA
:100ED4002A3D2A442A4B2A522A592A5F2A662A6D15
:100EE4002A742A7B2A822A882A8F2A962A9D2AA44F
:100EF4002AAB2AB12AB82ABF2AC62ACD2AD32ADA8B
:100F04002AE12AE82AEF2AF62AFC2B032B0A2B11C2
:100F14002B182B1F2B252B2C2B332B3A2B412B48F7
:100F24002B4E2B552B5C2B632B6A2B702B772B7E34
:100F34002B852B8C2B932B992BA02BA72BAE2BB56E
:100F44002BBC2BC22BC92BD02BD72BDE2BE52BEBA9
:100F54002BF22BF92C002C072C0D2C142C1B2C22DF
:100F64002C292C302C362C3D2C442C4B2C522C5917
:100F74002C5F2C662C6D2C742C7B2C822C882C8F53
:100F84002C962C9D2CA42CAA2CB12CB82CBF2CC68E
:100F94002CCD2CD32CDA2CE12CE82CEF2CF62CFCC9
:100FA4002D032D0A2D112D182D1F2D252D2C2D33FC
:100FB4002D3A2D412D482D4E2D552D5C2D632D6A36
:100FC4002D702D772D7E2D852D8C2D932D992DA073
:100FD4002DA72DAE2DB52DBC2DC22DC92DD02DD7AD
:100FE4002DDE2DE52DEB2DF22DF92E002E072E0DE5
:100FF4002E142E1B2E222E292E302E362E3D2E441C
:101004002E4B2E522E592E5F2E662E6D2E742E7B55
:101014002E822E882E8F2E962E9D2EA42EAA2EB191
:101024002EB82EBF2EC62ECD2ED32EDA2EE12EE8CC
:101034002EEF2EF62EFC2F032F0A2F112F182F1F01
:101044002F252F2C2F332F3A2F412F472F4E2F553B
:101054002F5C2F632F6A2F702F772F7E2F852F8C75
:101064002F932F992FA02FA72FAE2FB52FBC2FC2B0
:101074002FC92FD02FD72FDE2FE52FEB2FF22FF9EB
:1010840030003007300D3014301B3022302930301E
:101094003036303D3044304B30523059305F30665A
:1010A400306D3074307B30823088308F3096309D94
:1010B40030A430AA30B130B830BF30C630CD30D3D0
:1010C40030DA30E130E830EF30F630FC3103310A09
:1010D40031113118311F3125312C3133313A31413D
:1010E4003147314E3155315C3163316A317031777A
:1010F400317E3185318C3193319931A031A731AEB4
:1011040031B531BC31C231C931D031D731DE31E4EE
:1011140031EB31F231F932003207320D3214321B25
:101124003222322932303236323D3244324B32525C
:101134003259325F3266326D3274327B3282328897
:10114400328F3296329D32A432AA32B132B832BFD3
:1011540032C632CD32D332DA32E132E832EF32F60D
:1011640032FC3303330A33113318331F3325332C42
:101174003333333A33413347334E3355335C33637C
:10118400336A33703377337E3385338C33933399B7
:1011940033A033A733AE33B533BC33C233C933D0F2
:1011A40033D733DE33E433EB33F233F9340034072B
:1011B400340D3414341B3422342934303436343D61
:1011C4003444344B34523459345F3466346D34749B
:1011D400347B34823488348F3496349D34A434AAD6
:1011E40034B134B834BF34C634CD34D334DA34E112
:1011F40034E834EF34F634FC3503350A3511351848
:10120400351F3525352C3533353A35413547354E7F
:101214003555355C3563356A35703577357E3585BA
:10122400358C3593359935A035A735AE35B535BCF4
:1012340035C235C935D035D735DE35E435EB35F231
:1012440035F936003607360D3614361B3622362964
:1012540036303636363D3644364B36523659365F9E
:101264003666366D3674367B36813688368F3696DA
:10127400369D36A436AA36B136B836BF36C636CD14
:1012840036D336DA36E136E836EF36F636FC37034F
:10129400370A37113718371F3725372C3733373A82
:1012A40037413747374E3755375C3763376A3770BE
:1012B4003777377E3785378C3793379937A037A7F9
:1012C40037AE37B537BC37C237C937D037D737DE33
:1012D40037E437EB37F237F938003807380D38146C
:1012E400381B3822382938303836383D3844384BA2
:1012F40038523859385F3866386D3874387B3881DD
:101304003888388F3896389D38A438AA38B138B818
:1013140038BF38C638CD38D338DA38E138E838EF52
:1013240038F638FC3903390A39113918391E392588
:10133400392C3933393A39413947394E3955395CC1
:101344003963396A39703977397E3985398C3993FB
:10135400399939A039A739AE39B539BC39C239C937
:1013640039D039D739DE39E439EB39F239F93A0071
:101374003A073A0D3A143A1B3A223A293A303A36A5
:101384003A3D3A443A4B3A523A593A5F3A663A6DE0
:101394003A743A7B3A813A883A8F3A963A9D3AA41B
:1013A4003AAA3AB13AB83ABF3AC63ACD3AD33ADA57
:1013B4003AE13AE83AEF3AF63AFC3B033B0A3B118E
:1013C4003B183B1E3B253B2C3B333B3A3B413B47C5
:1013D4003B4E3B553B5C3B633B6A3B703B773B7E00
:1013E4003B853B8C3B933B993BA03BA73BAE3BB53A
:1013F4003BBC3BC23BC93BD03BD73BDE3BE43BEB76
:101404003BF23BF93C003C073C0D3C143C1B3C22AA
:101414003C293C303C363C3D3C443C4B3C523C59E2
:101424003C5F3C663C6D3C743C7B3C813C883C8F1F
:101434003C963C9D3CA43CAA3CB13CB83CBF3CC659
:101444003CCD3CD33CDA3CE13CE83CEF3CF63CFC94
:101454003D033D0A3D113D183D1E3D253D2C3D33C8
:101464003D3A3D413D473D4E3D553D5C3D633D6A02
:101474003D703D773D7E3D853D8C3D933D993DA03E
:101484003DA73DAE3DB53DBB3DC23DC93DD03DD779
:101494003DDE3DE43DEB3DF23DF93E003E073E0DB1
:1014A4003E143E1B3E223E293E303E363E3D3E44E7
:1014B4003E4B3E523E593E5F3E663E6D3E743E7B21
:1014C4003E813E883E8F3E963E9D3EA43EAA3EB15E
:1014D4003EB83EBF3EC63ECD3ED33EDA3EE13EE898
:1014E4003EEF3EF63EFC3F033F0A3F113F183F1ECE
:1014F4003F253F2C3F333F3A3F413F473F4E3F5507
:101504003F5C3F633F6A3F703F773F7E3F853F8C40
:101514003F933F993FA03FA73FAE3FB53FBB3FC27C
:101524003FC93FD03FD73FDE3FE43FEB3FF23FF9B7
:1015340040004007400D4014401B402240294030E9
:101544004036403D4044404B40524058405F406626
:10155400406D4074407B40814088408F4096409D60
:1015640040A440AA40B140B840BF40C640CD40D39B
:1015740040DA40E140E840EF40F640FC4103410AD4
:1015840041114118411E4125412C4133413A414109
:101594004147414E4155415C4163416A4170417745
:1015A400417E4185418C4193419941A041A741AE7F
:1015B40041B541BB41C241C941D041D741DE41E4BB
:1015C40041EB41F241F942004207420D4214421BF1
:1015D4004222422942304236423D4244424B425228
:1015E4004258425F4266426D4274427B4281428865
:1015F400428F4296429D42A442AA42B142B842BF9F
:1016040042C642CD42D342DA42E142E842EF42F5D9
:1016140042FC4303430A43114318431E4325432C0E
:101624004333433A43414347434E4355435C436347
:10163400436A43704377437E4385438C4393439982
:1016440043A043A743AE43B543BB43C243C943D0BE
:1016540043D743DE43E443EB43F243F944004407F6
:10166400440D4414441B4422442944304436443D2C
:101674004444444B44524458445F4466446D447467
:10168400447B44814488448F4496449D44A444AAA2
:1016940044B144B844BF44C644CD44D344DA44E1DD
:1016A40044E844EF44F544FC4503450A4511451814
:1016B400451E4525452C4533453A45414547454E4C
:1016C4004555455C4563456A45704577457E458586
:1016D400458C4593459945A045A745AE45B545BBC1
:1016E40045C245C945D045D745DE45E445EB45F2FD
:1016F40045F946004607460D4614461B4622462930
:1017040046304636463D4644464B46524658465F6A
:101714004666466D4674467B46814688468F4696A5
:10172400469D46A446AA46B146B846BF46C646CDDF
:1017340046D346DA46E146E846EF46F546FC47031B
:10174400470A47114718471E4725472C4733473A4E
:1017540047414747474E4755475C4763476A477089
:101764004777477E4785478C4792479947A047A7C5
:1017740047AE47B547BB47C247C947D047D747DEFF
:1017840047E447EB47F247F948004807480D481437
:10179400481B4822482948304836483D4844484B6D
:1017A40048524858485F4866486D4874487B4881A9
:1017B4004888488F4896489D48A448AA48B148B8E4
:1017C40048BF48C648CD48D348DA48E148E848EF1E
:1017D40048F548FC4903490A49114918491E492555
:1017E400492C4933493A49414947494E4955495C8D
:1017F4004963496A49704977497E4985498C4992C8
:10180400499949A049A749AE49B549BB49C249C903
:1018140049D049D749DE49E449EB49F249F94A003C
:101824004A074A0D4A144A1B4A224A294A2F4A3671
:101834004A3D4A444A4B4A524A584A5F4A664A6DAC
:101844004A744A7B4A814A884A8F4A964A9D4AA4E6
:101854004AAA4AB14AB84ABF4AC64ACD4AD34ADA22
:101864004AE14AE84AEF4AF54AFC4B034B0A4B115A
:101874004B184B1E4B254B2C4B334B3A4B414B4790
:101884004B4E4B554B5C4B634B6A4B704B774B7ECB
:101894004B854B8C4B924B994BA04BA74BAE4BB506
:1018A4004BBB4BC24BC94BD04BD74BDE4BE44BEB42
:1018B4004BF24BF94C004C074C0D4C144C1B4C2276
:1018C4004C294C2F4C364C3D4C444C4B4C524C58B0
:1018D4004C5F4C664C6D4C744C7B4C814C884C8FEB
:1018E4004C964C9D4CA44CAA4CB14CB84CBF4CC625
:1018F4004CCD4CD34CDA4CE14CE84CEF4CF54CFC61
:101904004D034D0A4D114D184D1E4D254D2C4D3393
:101914004D3A4D414D474D4E4D554D5C4D634D6ACD
:101924004D704D774D7E4D854D8C4D924D994DA00A
:101934004DA74DAE4DB54DBB4DC24DC94DD04DD744
:101944004DDE4DE44DEB4DF24DF94E004E074E0D7C
:101954004E144E1B4E224E294E2F4E364E3D4E44B3
:101964004E4B4E524E584E5F4E664E6D4E744E7BED
:101974004E814E884E8F4E964E9D4EA44EAA4EB129
:101984004EB84EBF4EC64ECC4ED34EDA4EE14EE864
:101994004EEF4EF54EFC4F034F0A4F114F184F1E9A
:1019A4004F254F2C4F334F3A4F414F474F4E4F55D2
:1019B4004F5C4F634F6A4F704F774F7E4F854F8C0C
:1019C4004F924F994FA04FA74FAE4FB54FBB4FC249
:1019D4004FC94FD04FD74FDE4FE44FEB4FF24FF983
:1019E400500044313233343536373839302A2341C4
:1019F400424320202020202020202020202020209E
:101A040020202020202020202020202020202020D2
:101A1400202020494C4C4547414C20454E545259B6
:101A2400202020204F5554505554204C4556454CA9
:101A3400202020202020202020202020205241541B
:101A4400494F20202020202053494E4520574156FD
:101A54004520465245513A20202020202020202095
:101A6400487A20204F5554204F462052414E474536
:021A7400202030
:1056890030281CE53E540F9019E6939000A2F012C1
:105699005348754B3212618E12610BC228800CE59A
:1056A9004B700890008FF090009FF030291BE53C6B
:1056B900540F9019E6939000A1F01252E4754C3200
:1056C90012618E12610BC22922E54C70089000907C
:0656D900F090009EF0229B
:06618E00900094E004F013
:106194009000A4E014600A14600A240270090261E9
:0861A400AC025EEF124FFE2277
:1061AC003028099000A2E0B42A02800A30290D9010
:0D61BC0000A1E0B42A069000A4E004F02247
:105EEF003028099000A2E0B43502800A30291E90B4
:105EFF0000A1E0B4351790003D740AF090000E74C5
:105F0F0020F0A3F0A3F09000A4E004F022E49000AE
:035F1F00A4F022C9
:104FFE0030282D9000A2E0FF12626F50239000A285
:10500E00E0FF90003DE0FE04F074042EF582E434DF
:10501E0000F583EFF090003DE0D3940C4040802EDD
:10502E003029369000A1E0FF12626F502C9000A143
:10503E00E0FF90003DE0FE04F074042EF582E434AF
:10504E0000F583EFF090003DE0D3940C4010124930
:0F505E000512624FE4FF022AC2E49000A4F02280
:1049050090000FE0540F75F00AA4FDACF090000E76
:10491500E0540F75F064A42DFFE5F03CFE90001007
:10492500E0540F7C002FF565EC3EF564D3E5659406
:1049350000E564648094804048D3E56594FFE564B0
:1049450064809480503B7BFF7A1A7926125F8C7BBA
:10495500FF7A1A7936125FBD7F12122AC290000EB5
:10496500E0FF122A9390000FE0FF122A93900010A7
:10497500E0FF122A93856536755903E55970FC8069
:10498500197BFF7A1A7916125F8C7BFF7A1A7906E2
:10499500125FBD755903E55970FC7BFF7A1A79469C
:1049A500125F8C7BFF7A1A7956125FBDE49000A4E2
:0149B500F011
:0149B60022DE
:10610B003028099000A2E0B42302800A30291290B3
:10611B0000A1E0B4230B122C3A12624FE4FF122AB7
:02612B00C2228E
:102C3A0075640075650FAF6574512FF582E4340031
:102C4A00F583E064236003022E2774502FF582E493
:102C5A003400F583E0FF12626F4003022E277BFFE8
:102C6A007A1A7946125F8C7BFF7A1A7956125FBDFF
:102C7A007F1B122AC274502565F582E43400F5835D
:102C8A00E0FF540F756600F567122A93744F2565A5
:102C9A00F582E43400F583E0FF12626F4003022EEE
:102CAA0006AD65744F2DF582E43400F583E0540FC8
:102CBA0075F00AA4FFAEF074502DF582E43400F5E5
:102CCA0083E0540F7C002FF567EC3EF5667F1A12FD
:102CDA002AC2744F2565F582E43400F583E0FF12B9
:102CEA002A93744E2565F582E43400F583E0FF12D9
:102CFA00626F4003022E06AD65744F2DF582E434EF
:102D0A0000F583E0540F75F00AA4FBAAF0744E2D67
:102D1A00F582E43400F583E0540F75F064A42BFFC8
:102D2A00E5F03AFE74502DF582E43400F583E05460
:102D3A000F7C002FF567EC3EF5667F19122AC274E4
:102D4A004E2565F582E43400F583E0FF122A937478
:102D5A004D2565F582E43400F583E0FF12626F4089
:102D6A0003022E06AB65744D2BF582E43400F5831D
:102D7A00E0540FFF7E007C037DE81246D6AC06AD18
:102D8A0007744E2BF582E43400F583E0540F75F096
:102D9A0064A42DFDEC35F0FC744F2BF582E434006D
:102DAA00F583E0540F75F00AA42DFFE5F03CFE749C
:102DBA00502BF582E43400F583E0540F7C002FF5A4
:102DCA0067EC3EF5667F18122AC2744D2565F582B6
:102DDA00E43400F583E0FF122A93D3E56794B8E55B
:102DEA0066940B40177BFF7A1A7966125F8C7BFF19
:102DFA007A1979F6125FBDE4FF022AC2E56725E077
:102E0A00FFE56633FE74742FF58274023EF583E49F
:102E1A0093F508740193F509D231D21322E56515A9
:102E2A006570021564D3E5659400E5646480948056
:052E3A004003022C40E2
:012E3F002270
:10624F00E4900094F07F109000517420F0A3DFFCD5
:01625F00221C
:10614E0075081A7509ABD231D2137BFF7A027954D6
:10615E00125F8C7BFF7A027965125FBDE4FF022A23
:01616E00C26E
:105A83002A2A3132333435362A2A2A2A3132333418
:105A930035302A2A44313233343536373839302ACF
:105AA30023414243202056455253494F4E20312E25
:105AB300302020202053494E452047454E45524132
:045AC300544F5220CA
:104A6700302825C228E53E540F905A97939000A20C
:104A7700F0125348754B32900094E004F030011463
:104A8700125E52125CFF800CE54B700890008FF0AD
:104A970090009FF030293DC229E53C540F905A976A
:104AA700939000A1F01252E4754C32900094E00408
:104AB700F0301C03200006201C06300203125CC4E1
:104AC700301C03200003201C03125E1D201C111242
:104AD7005F22800CE54C7008900090F090009EF0EB
:104AE7003023193003221252E4754D321262F390CB
:104AF7000093EFF0C223125D3A025E87E54D70081E
:094B0700900091F09000A0F02252
:105E1D00900090E0FF04F0EF905A8393FF9000A163
:105E2D00E0FEEF6E6011EEB42A089000907401F060
:105E3D008005E4900090F0900090E0B40A06E4F044
:055E4D00D21FD22A2241
:105E520090008FE0FF04F0EF905A8393FF9000A22E
:105E6200E0FEEF6E6011EEB42A0890008F7401F02C
:105E72008005E490008FF090008FE0B40A06E4F011
:055E8200D21ED22A220D
:105E8700900091E0FF04F0EF905A8393FF90009306
:105E9700E0FEEF6E6011EEB42A089000917401F0F5
:105EA7008005E4900091F0900091E0B40A06E4F0D8
:055EB700D220D22A22D6
:105CC40090009EE0FF04F074952FF582E43400F513
:105CD40083E0FF9000A1E0FEEF6E6011EEB42308B4
:105CE40090009E7401F08005E490009EF090009E68
:0B5CF400E0B40906E4F0D21FD21D222C
:105CFF0090009FE0FF04F074952FF582E43400F5D7
:105D0F0083E0FF9000A2E0FEEF6E6011EEB4230877
:105D1F0090009F7401F08005E490009FF090009F29
:0B5D2F00E0B40906E4F0D21ED21D22F1
:105D3A009000A0E0FF04F074952FF582E43400F59A
:105D4A0083E0FF900093E0FEEF6E6011EEB423084B
:105D5A009000A07401F08005E49000A0F09000A0EB
:0B5D6A00E0B40906E4F0D220D21D22B4
:105F2200900092E0FF04F0EF905A8D93FF9000A151
:105F3200E0FEEF6E6011EEB42A089000927401F058
:105F42008005E4900092F0900092E0B40A04E4F03C
:035F5200D22B222D
:106046009000957423F0A3F0E4FF746D2FF582E4BD
:106056003400F583E0FE74972FF582E43400F5836F
:0C606600EEF00FBF06E490009D7423F0E4
:01607200220B
:105DAE001229F07BFF7A5A79B7125F8C7BFF7A5AF1
:105DBE0079A7125FBD752E147F10900051E4F0A3E9
:105DCE00DFFC7F10E52E70FC122ADC122AEB7F011D
:085DDE00122AC2E4900094F0C7
:015DE600229A
:1052E400900094E0FED3940F50129000A1E0FF745C
:1052F400512EF582E43400F583EF80437F01122AB6
:10530400C2E4F56474522564F582E43400F583E064
:10531400FF74512564F582E43400F583EFF0745191
:105324002564F582E43400F583E0FF122A930564D2
:10533400E564C3940F40CD9000A1E0FF900060F0BD
:03534400122A9397
:015347002243
:10534800900094E0FED3940F50129000A2E0FF74F6
:10535800512EF582E43400F583EF80437F01122A51
:10536800C2E4F56474522564F582E43400F583E000
:10537800FF74512564F582E43400F583EFF074512D
:105388002564F582E43400F583E0FF122A9305646E
:10539800E564C3940F40CD9000A2E0FF900060F058
:0353A800122A9333
:0153AB0022DF
:0362F3007F012206
:030000000262B0E9
:0C62B000787FE4F6D8FD75819B02546BEA
:1046A900BB010CE58229F582E5833AF583E02250C6
:1046B90006E92582F8E622BBFE06E92582F8E22210
:0D46C900E58229F582E5833AF583E493222A
:1046D600EF8DF0A4A8F0CF8CF0A428CE8DF0A42EF8
:0246E600FE22B2
:1046E800BC000BBE0029EF8DF084FFADF022E4CCB6
:1046F800F875F008EF2FFFEE33FEEC33FCEE9DEC7F
:10470800984005FCEE9DFE0FD5F0E9E4CEFD22EDC4
:10471800F8F5F0EE8420D21CFEADF075F008EF2F0E
:10472800FFED33FD4007985006D5F0F222C398FDFF
:054738000FD5F0EA229C
:10473D00A3F8E0C5F025F0F0E5821582700215832F
:06474D00E0C838F0E8228C
:0C475300A42582F582E5F03583F5832271
:10475F00D083D082F8E4937012740193700DA3A3E9
:10476F0093F8740193F5828883E4737402936860FD
:06477F00EFA3A3A380DFFD
:00000001FF
